:020000020000FC
:040000000C948200DA
:1001000000EC05BFC0EDD0E000E003500DBF01E002
:1001100000400EBF0E943601002309F424D0E0E61F
:10012000F0E000E110E00E94C512E0E0F0E000E045
:1001300010E040E050E00E94B712E4E0F1E00CE58E
:1001400013E00E94C512E8E3F2E000E011E044E0B1
:1001500050E00E94B712EAE6F1E000E614E040E069
:0A01600050E00E94B7120C94380121
:04026C0001E0089510
:100270000E946805002319F40E945B03FDCFF894E7
:0C0280000E94730178940E949001FDCF51
:10016A000A53494F32494445207665722E20322E71
:10017A00312028632932303032204D4D536F667456
:02018A000A0069
:10028C005798E2E6FF2700831183E0E6F083F183C1
:10029C00E4E6F083579A089519B71D7F19BF0093B0
:1002AC00060209B7026009BF089509B70D7F09BF9F
:1002BC0000910602002311F0002701C001E019B7DC
:1002CC00126019BF08950EEFE7DF04E010E0D8DFED
:1002DC00949A01E00093040208958C9A909A0FE08E
:1002EC0009B908E90AB98A98929A0FEC02BF05E09D
:1002FC0003BF09B7026009BFE6CF202F312F015091
:10030C001040232B11F00000F8CF08955D9BFECF19
:10031C000CB908950E94D912A4E0B1E0C6DF002305
:10032C0009F0D1DF00910402ECE3F2E00C945A12D4
:10033C00829BA6C00EEFB0DFEA2FFB2F41810A2F64
:10034C001B2F0E948805002309F499C000270093F5
:10035C000502B0D0E457FE4FC895002009F48DC0BB
:10036C00A9D0E457FE4FC895EA2FFB2F0181001648
:10037C0021F5A0D0AAD0002901F155270091050242
:10038C00112746E00E94C411E02FF12F9ED0E02FE0
:10039C00F02D42E650E00A2F1B2F0995002369F03F
:1003AC0089D0E157FE4FC89500920402E2E6FF2780
:1003BC000081118165DF949863C00091050203955B
:1003CC00C6CF08EC10E06BD009F44EC073D0E057E8
:1003DC00FE4FC89570D009F447C003E497DF07E0DF
:1003EC0036C042C041C00AEF10E087DF4ED030F576
:1003FC00E0E6008111810C5F1E4FE02FF12F008190
:10040C0085DFFF2704E610E0E0E62081318166D02D
:10041C003327E4E6FF274081240F331F3150E0E6F9
:10042C002081318118F05AD0239501C057D0E02F8C
:10043C00F12F0081020F008357D0D8CFE4E6008162
:10044C001DC04AD002E028DF01E460DF04E0009325
:10045C00040216C000ED17E022D031F02BD0E0578B
:10046C00FE4FC89528D021F405E408C035D04ED0F5
:10047C0003E404C004EF11E040DF0EE447DF23DFA8
:10048C00E4E00C94EA1202E007DFE0E6FF270081CB
:10049C001181E2E6208131810217130708952DDFC7
:1004AC0035D02AD0E057FE4FC895002D3196C8950F
:1004BC000029089521C0002D3196C895E02FF02D0C
:1004CC0004E011E0099500230895E357FE4FC89509
:1004DC00002D3196C895089508EC1BC02C5F3E4F3B
:1004EC00E22FF32F20810895E0E6008111810F5F48
:1004FC001F4F00831183089500910502112746E0D8
:10050C0050E00E94C411E02FF12F089501E4FEDEAB
:10051C000AEF10E0F2CE0A921A922A923A920A93B9
:10052C001A932A933A934A935A936A937A93EA9337
:10053C00FA93FFB7FA938A938CB1829919C0009100
:10054C0004020130A9F49FDF50F441D0082F08F0C9
:10055C000395E22FF32F1081100F108309C0E4E6EE
:10056C000081081711F402E001C008E000930402B6
:10057C00829B1BC0009104020430B9F484DF48F460
:10058C0026D008F08395E22FF32F0081080F00830B
:10059C000CC00EEF81DEE4E6FF270081081711F492
:1005AC0005E001C009E0009304028991F991FFBFB5
:1005BC00F991E991799169915991499139912991DF
:1005CC0019910991399029901990099018958CDFFF
:1005DC00015010400C5F1E4FE02FF12F8083E4E69A
:1005EC00FF2724E630E0082F11274081040F1F1F3E
:1005FC00115008950A93EA93FA93FFB7FA93009176
:10060C0006020E3F49F000910602002329F00091EA
:10061C0006020150009306020FEC02BFF991FFBFD6
:08062C00F991E991099118957B
:10023C000200460209009E01270246023002E70135
:08024C00F901450240023C02E9
:04002C000C9400032D
:040034000C94910295
:10063400402F512F622F732F015010402040304023
:10064400452B462B472B11F00000F2CF089529D0FB
:100654000E941D12742E7394082F192F2A2F3B2FDA
:10066400E42D1FD00E941D12E42D1ED00E941D12E5
:10067400642E2A2F3B2FE42D0381148142815527B8
:100684000E94C411402F512F66277727082F192F56
:100694000E941D12402E512E062D0F700056602E02
:1006A40008954381548102C04281552766277727E4
:1006B400089500EA16E821E030E0BADFAD9800E4DE
:1006C4001DE023E030E0B4DFAD9A089531E040E866
:1006D4001127332339F0202F232309F0142B330F50
:1006E4004695F7CF012F08959A938A93902F042F5C
:1006F400852FECDF1FEF1ABB17BBF89415B3107EE0
:10070400192B15BBAF980BBB88BBAF9A000005B380
:100714000F6105BB78940FEF0ABB0BBB07BB08BB8B
:100724008991999108959A938A9311271ABB1FEF7F
:100734001BBB112717BB1FEF18BBF89415B3107E12
:10074400102B15BBAE980000AE9A09B386B315B34F
:100754001F6115BB78941FEF1ABB1BBB17BB18BBDB
:10076400B5DF182F8991999108950E94DA12A02F6C
:1007740080E197E2AA2339F00197082F092B19F495
:10078400AD98002705C00DE1CEDF00309CF301E0F9
:10079400E3E00C94EB1211D0882339F011970A2F5F
:1007A4000B2B19F4AD98002705C00DE1BCDF06FF43
:1007B400F3CF01E0E4E00C94EA120E94D912802FF6
:1007C400A0E1B7E20895F9DF882339F011970A2FE1
:1007D4000B2B19F4AD98002705C00DE1A4DF03FF2E
:1007E400F3CF01E0E4E00C94EA120DE19CDF00FF9A
:1007F40003C0AD9801E00895AD9A0027089529D06B
:10080400B8F0E42DF52D01850030042F2CF0152FC0
:10081400262F372F1CDF01C02FD015D049F035D03B
:1008240041E20AD029F0E1DF002311F401E001C024
:100834000027E8E00C94E61250E00DE155DF01E0FA
:10084400C2DF0023089505E06EDF01E08EDF0023A0
:1008540008950E94D512402E512E842F952FA62F35
:10086400B72FE02FF12F05811681278130850417DA
:100874001507260737070895702E492E5A2E6B2E1A
:100884000FE0602200EE600E0895462D552709E121
:100894002BDF41E050E009E027DF472D55270DE02D
:1008A40023DF442D552701E11FDF452D50E005E1ED
:1008B4001BCFCFDF90F0E42DF52D01850030042F00
:1008C4002CF0152F262F372FC2DE01C0D5DFBBDF5A
:1008D40021F0DBDF41E3B0DF11F4002701C001E0C8
:1008E400E8E00C94E61215D08ADF002371F00A2F99
:1008F4001B2F1197012B01E049F015DFE82FF92F89
:10090400019311938E2F9F2FF2CF0027E8E00C94D0
:10091400EA120E94D912802F912F042F152F4C8197
:100924005D816E817F81A0E0B1E00895F2DFC1DFD7
:10093400002381F00A2F1B2F1197012B49F0E82F78
:10094400F92F419151918E2F9F2F01E0CDDEF2CFEF
:1009540001E001C00027E8E00C94EA120E94D712DB
:10096400A02FB12F0027EA2FF12F008301830283E8
:10097400038304830583068307830087018705E0D7
:10098400D2DE40EA50E009E1AFDE01E0EEDE002312
:1009940009F471C04CEE50DF09F46DC026DF00236A
:1009A40009F069C04424552401E0501608F040C001
:1009B400BADE802F912F042D152DE4E5F2E00C947E
:1009C4005E12EA2FFB2F808391832EC0EA2FFB2F28
:1009D40082832AC0EA2FFB2F8383948325C091FF4F
:1009E40023C0EA2FFB2F0185006801871DC0EA2F71
:1009F400FB2F01850030C4F4222785839683278347
:100A0400208712C0EA2FFB2F018500306CF41127D8
:100A14004581568167817085410F511F681F791F79
:100A240045835683678370870FEF401A500ABCCF03
:100A3400EA2FFB2F01850030E4F000811181222789
:100A4400332732DE0E94F811EA2F2BDE0E94F811C0
:100A5400EA2F058316832783308705811681278132
:100A64003085015010402040304005831683278391
:100A7400308701E001C00027E6E00C94E8129A9365
:100A84008A93802F912F0FEF0ABB0BBB07BB08BBC8
:100A940004BB0FE105BBAE9AAF9AAD9840EA50E0B3
:100AA40009E122DE002761DE002775DE00E513EC94
:100AB40020E030E0BDDD082F192F50DF002311F4B2
:0C0AC400002701C001E08991999108957C
:100254000001011605E30402E80403EC042BF10495
:070264000BF904010405FB86
:100AD0008D988E988F98959A969A979A00B3003031
:100AE0008B9A14F0939801C0939AE5E6FF27F08360
:100AF0000E940D11002311F40027089500B3003067
:100B00000CF08B9A939A01E0E5E6FF2700830895A5
:100B1000E02FF12F2081213711F4859B07C0E02FB2
:100B2000F12F2081223701F5859B1EC04131C1F094
:100B30004231B1F04631A1F0433191F0443181F0BE
:100B4000453171F0473161F0483151F0493141F0A0
:100B50004A3131F04B3121F04C3111F04D3111F46B
:100B600001E0089500270895E02FF12F208121331F
:100B700018F02081293310F00027089520B3203089
:100B80003CF4E02FF12F2081213311F40027089548
:100B900086990EC0E02FF12F2081213311F422E33A
:100BA00006C0E02FF12F2081223311F421E32083AE
:100BB000E02FF12F008100530E947A0E012B11F0DB
:100BC00001E0089500270895E02FF12F20812053A0
:100BD00020930702238102810093080220930902D7
:100BE000009107020E947A0E2091080230910902BA
:100BF0000217130708950CD00CE010E0E42FF52F36
:100C000000831183009107020E947A0E012B089540
:100C1000E02FF12F008100530093070208951DD0AB
:100C200031F0D2DF20F0022F132F032B11F4002715
:100C300011C0E22FF12F319738F0E22FF12F3497C6
:100C400018F400E810E001C015D0E82FF92F008358
:100C5000118301E08991999108959A938A93842F41
:100C6000952FE5E6FF272081222308959A938A9302
:100C7000802F912F009107020C94650E02D00C94E6
:100C8000FC0F1A930A9340910802509109020091B7
:100C900007020895E2DF31F097DF20F0022F132FD3
:100CA000032B11F4002711C0E22FF12F319738F0F8
:100CB000E22FF12F349718F400E810E001C0DADFDA
:100CC000E82FF92F0083118301E08991999108950C
:100CD000D8DF0C94820F9CDF04E00FD00AD0012BE8
:100CE00011F400270895E5E6FF27008108958E2F6F
:100CF0009F2F009107020C947A0E10E0E42FF52F3D
:100D0000008311830895B2DF0030114011F400E335
:100D100001C000E1E82FF92F01930FEF019300EEDE
:100D200001930027008301E089919991089563DF81
:100D3000D1F600270895D7CF9A938A93802F01E0A8
:100D4000E82FF12F019300E10193D1DFE82FF92F74
:100D50001193CDDFE82FF92F0193002701938E2FF8
:100D60009F2F88DF0030114041F40CE0E82FF92F6D
:100D7000019301E00193002707C008E0E82FF92F55
:100D800001930027019300E8019300E4019309E433
:100D9000019304E4019305E4C5CF2DDF09F0A3CF4F
:100DA00000270895A0CF9A938A93E02FF12F828194
:100DB000982F0381802F9DDF0817190711F0002756
:100DC00001C001E08991999108959A938A93842FA3
:100DD000952F1EDF0E94650EE82FF92F00831183E7
:100DE00000811181012B11F4002703C0E5E6FF27E4
:100DF000008189919991089539DF025010402FEFB9
:100E0000E82FF92F21932193202F312F01501040EB
:100E1000232B09F488CF2227F6CF85CF1A930A9384
:100E20000027E42FF52F00830183229608951A935B
:100E30000A93002722960895E02FF12F0281009354
:100E400007020FE05ADF009107020C945D0E402F5D
:100E5000512F009107020C94820DEECF402F512F9D
:100E6000009107020C94B10D1A930A930FE045DF2D
:100E7000E5E6FF270081229608950C94560DF4CFE5
:100E80000C94730D21E030E0E42FF52F20833183A3
:100E9000E02FF12F02810C943F0E2FEFE02FF12F66
:100EA000208321CF1A930A9301E0E1CF2FEFE02FA7
:100EB000F12F20830C948E0E1A930A930AE0D7CF59
:100EC0000E94F80E01E008951A930A9304E0CFCF30
:100ED0000E94FE0E01E008951A930A930FE0C7CF17
:100EE0000C94F80CF9CF0C940D0DF6CF0C941F0D4B
:100EF000F3CF0E942F0D01E00895EECF9A938A93CD
:100F0000802F912F0E947C10002329F0082F192F89
:100F10000E942F0D08CF0FE010E01A930A93442788
:0C0F20005527082F192F0E943013FDCE1A
:10018C00536B06068306500F06033E06570F0603F5
:10019C003E06524A060668064E9706069C064FCD4A
:1001AC000603D30621E50606FC063F0E07061707D5
:1001BC00111C07062707122D07032E0713340706F9
:1001CC003D07143F0706400716520706560715420F
:1001DC0007064D07175C07066007186407066807D3
:1001EC00196C070670071A72070673071B7507034D
:1001FC0076071C78070679071D7D07067E07000029
:04020C0000010000ED
:100F2C000E94D912802F912FA22FB32FE0E0F1E075
:100F3C0057D05FD0A1F0BA93AA939A938A9346E6BE
:100F4C0055270AE012E00E947504002311F40027D3
:100F5C0007C0E0E0F1E080839183A283B38301E0DA
:100F6C00E4E00C94EA120E94D912802F912FA42F46
:100F7C00B52F49C022273327015010402040304064
:100F8C00442D552D50D0082D57D0E65FFB4F0081D6
:100F9C00118122813381800F911FA21FB31F0895ED
:100FAC00041B150B260B370B4091540455273BD0D3
:100FBC008E5F9F4FAF4FBF4F0895802F912FA22F61
:100FCC00B32F823000E01007200730070895802FE0
:100FDC00912FA22FB32F0F3F1F4F0895EAE0F4E09B
:100FEC00008111812281338108958F5F9F4FAF4F14
:100FFC00BF4F80179107A207B30708959A938A935E
:10100C00802F912F089540E75AE027D200230895AE
:10101C00662777270E94F811E2E4F4E045815681B7
:10102C00678170850895662777270E941D12802F8F
:10103C00912FA22FB32F0895112747E050E00E9463
:10104C00C411E02FF12F08953A932A931A930A931F
:10105C0046E655270AE012E00C9498040E94D91237
:10106C00802F012F122F232F33270ED019F4002796
:10107C00112705C0E82FFF2711D0008111812227ED
:10108C003327E4E00C94EA12E2E4F4E0418152816B
:10109C006381748108D044DF00230895EE0FFF1F95
:1010AC00E65FFD4F0895040F151F261F371F089587
:1010BC000E94D912802F47E00E941412E5DF29F418
:1010CC00002711272227332708C0E82FEF77FF27A7
:1010DC00EE0FFF1FE3DF84DF3F70E4E00C94EA12B5
:1010EC000E94D512602E712EE02FF12F79DF5FD088
:1010FC0028F4E62DF72D74DF53DF01C053D04424C0
:10110C00552400914204045029F0025019F0065065
:10111C00D9F036C0082F192F2A2F3B2F9FDF402FD5
:10112C00412B422B432B61F14FEF441A540A0F3FD2
:10113C00140740E02407340711F057DF09F547DFA7
:10114C002040304039F719C0082F192F2A2F3B2F78
:10115C00AFDF402F412B422B432B91F04FEF441A22
:10116C00540A0F3F140724074FE0340711F03DDFFA
:10117C0039F42DDF2F4F3F4039F7042D152D07C0C3
:10118C00E62DF72D06810062068300271127E8E083
:10119C000C94E6120E94D512602E712E442E552E00
:1011AC0011D005C082E090E0A0E0B0E00895E2E448
:1011BC00F4E04581568167817085401751076207BD
:1011CC0073070895E5E5F4E00281138124813581EC
:1011DC0008950E94D912802F912FA42FB52F40D0A3
:1011EC0046815781608571853CD0B0F500915F04D4
:1011FC00112745E00E94D411065F1D4F0093550442
:10120C001093560400915F040031E0F4DDDF32D01E
:10121C0011F4002722C000915F04039500935F0432
:10122C00082F192FEA2FFB2F0995002311F001E04D
:10123C0014C0E5E5F4E000811181005E1F4F0083CE
:10124C001183E0CF002700935F04BEDF0F5F1F4FB9
:10125C002F4F3F4F12D0C3CF02E0E4E00C94EA12C0
:10126C00B1CF04171507260737070895082F192F34
:10127C002A2F3B2F10CFE5E5F4E002831383248360
:10128C0035830895A6DF002339F00A9519F00A95E5
:10129C0019F002C001E00895002708950E94D912A8
:1012AC0024D028D0E8DF14D0428153816481758129
:1012BC0028D00683178320873187002700935F048B
:1012CC00482F592F0A2F1B2FDDDFE4E00C94EA1274
:1012DC000091540411274091530455270E94C411C6
:1012EC00212F210F220B322F0895A02FB12F842FE5
:1012FC00952F0895E2E4F4E0018512852385348569
:10130C000895D1CE47DF10F44BDE01C04BDF4FD038
:10131C0039F00A9519F00A9529F004C001E011C0C2
:10132C0000270FC0082F192F2A2F3B2F97DE45DEE1
:10133C0010F00AD001C0DEDF11D000E0A007B0072A
:10134C0031F7E8E00C94E612082F025010402040D0
:10135C0030404091540455275BDEA5CE8CDF0091C4
:10136C0054041127222733274281538164817581CC
:10137C009ADE06831783208731878F3F0FEF900704
:10138C000895442D552D0E94E21141505040042FD8
:10139C00152F462D572D0C94C411442D552D0E94FC
:1013AC00E211452B082F192F2A2F3B2F0895442D7E
:1013BC00552D062D172D0DDF0023089504D0A2DF27
:1013CC00E4E00C94EA120E94D912E2E4F4E0058401
:1013DC00168427843088E5E5F4E0028213822482A7
:1013EC003582009054041124222433248281938169
:1013FC00A481B581080E191E2A1E3B1E0682178277
:10140C0020863186222720935F040895C3DE10F4D2
:10141C00C7DD01C0C7DECBDFB9F00A9519F00A951C
:10142C0021F003C001E011C00FC0082F192F2A2F83
:10143C003B2F3EDEC2DD10F087DF01C05BDF8EDFAD
:10144C00A0070FE0B00739F70027E8E00C94E6128C
:10145C00BADFDCDFE4E00C94EA120E94D91220918E
:10146C004204245029F0225019F0265039F008C0BB
:10147C000BD011F413DF05C0A1DF03C0E9DF01C0FD
:10148C000027E4E00C94EA12E2E4F4E0058416840C
:10149C002784308881859285A385B4850816190622
:1014AC002A063B0608950E94D9122091420424502A
:1014BC0029F0225019F0265039F008C0E5DF11F45C
:1014CC00E1DE05C01FDF03C0A1DF01C00027E4E09F
:1014DC000C94EA120E94D112602E712EC1D0062DEE
:1014EC00172D0E943013BDD0828C938C04891589E2
:1014FC00A02EB12E0081053E09F48AC003850E7D15
:10150C0009F086C0B3D0012B022B032B09F480C049
:10151C00B2D04DE152E0B1D0C1F4A3D0A7D001308C
:10152C0012402040304008F073C008E0E62DF72D43
:10153C000687002711270487058702E0801691068D
:10154C00A106B10608F06DC075C095D040E152E01F
:10155C0094D009F05DC085D0038500FF05C0E62D51
:10156C00F72D06850460068792D018F099D0EDDE31
:10157C0001C0C0DE7FDE09F44BC00AE012E020910E
:10158C000A0230910B022639324029F0E62DF72D54
:10159C00268520612687E02FF12F2481358120308C
:1015AC00314029F4E62DF72D068500640BC0E02FA1
:1015BC00F12F048115810038104029F0E62DF72D0C
:1015CC00068500610687E62DF72D068506FF04C00B
:1015DC00442401E0502E03C000E8402E552440DE88
:1015EC0049DEB1F03ED0848D958DA68DB78D80519E
:1015FC009040A040B0402AD0452B462B472B51F0B1
:10160C00E091550433D0013011402040304010F0AF
:10161C00002719C01BD0E62DF72D0487158737D06E
:10162C0048F00EEF800E0FEF901EA01EB01E38D0AB
:10163C0090DE01C05FDEE62DF72D37D0062D172D7D
:10164C000E94191301E0ECE00C94E212082F192F00
:10165C002A2F3B2F442D552D662777270C941D12CE
:10166C002AC0E0915504F09156040895048D158D0F
:10167C00268D378D089503E026C0009155041091F6
:10168C005604085F1F4F0E942A11012B089502E097
:10169C00801600E09006A006B00608950E9419136B
:1016AC00082D192D2A2D3B2D08950087118722878F
:1016BC00338708D00CC00FE010E01A930A9344272C
:1016CC005527089508E010E01A930A930895409165
:1016DC00550450915604089546DC51F013D01BD09C
:1016EC000E942A11012B11F401E003C00DD0B1F7B7
:1016FC000027E4E00C94EA12E5DF0DD00E94F5120D
:10170C00012B089508E0DFCF40E75AE0082F192F8E
:10171C00CADE002308954A2F5B2F082F192F089536
:10172C0022DC31F0E9DF11F401E003C0EDDFD1F789
:10173C000027E4E00C94EA1216DC31F0DDDF11F442
:10174C0001E003C0E1DFD1F70027E4E00C94EA12DA
:10175C000ADC79F0E82FF92F18D0EA2FFB2F408103
:10176C005181628173817DDD11F401E003C0CCDF16
:10177C0089F70027E4E00C94EA12E82FF92F219363
:10178C008E2F9F2FE02FF12F089500851185228534
:10179C00338508959A938A932F9700271127222730
:1017AC00332768DD09F483C02AE032E0EAE0F2E096
:1017BC00E250FE4F0081118105351A4A09F077C0BD
:1017CC0022543E4FE22FF32F0081003809F06FC0F6
:1017DC00048100934204D9DF4DDD09F468C08AE02E
:1017EC0092E000914204045029F0025019F0065086
:1017FC0049F15DC061D04385548578D041875287CB
:10180C0063877487458756876787708BE82FF92F16
:10181C000681178144E00E94DB11177F409154042C
:10182C0055270E94E2110093530452DDE2E4F4E0E8
:10183C00418552856385748564DD05831683278312
:10184C00308733C039D0418D528D50D0458356836B
:10185C006783708701E000935304E82FF92F01A1EF
:10186C0012A123A134A1023010402040304030F0AE
:10187C0001A112A123A134A168DD01C03BDD0187C8
:10188C00128723873487058716872787308B34DDAB
:10189C00088719872A873B8700270C870D8746D036
:1018AC00202F212B11F00093530401E001C00027DD
:1018BC002F968991999108950B96E82FF92F4189CC
:1018CC005289638974890381148122273327400F3D
:1018DC00511F621F721FE2E4F4E041835283638361
:1018EC007483E82FF92F0581112708950E94C411E4
:1018FC00228120935404418952896389748903801D
:10190C001480400D511D631F731F2227400F511F60
:10191C00631F721FE2E4F4E008950C2F1D2F085F83
:10192C001F4F1A930A9341E252E008950C2F1D2F7A
:10193C00085F1F4FD5CB9A938A93992781E0883003
:10194C0050F4082F0DD0E05FFB4F008100300CF4F9
:10195C0093958395F4CF092F899199910895082D2A
:10196C006BCB37D07EDE028D138D44895589242FA5
:10197C00352F4081453E59F0438544FF08C0448DC6
:10198C00558D668D778D452B462B472B11F00027F7
:10199C001DC044275527E82FF92F4487458702306F
:1019AC0014072407340748F0025010402040304000
:1019BC00409154042DDBA5DC01C09CDCE82FF92FF1
:1019CC0074DE082F192F0E94191301E08991999147
:1019DC0008959A938A93802F912F6DDE082F192FDB
:1019EC000C9430130BDB47EB5CE037DD002331F05C
:1019FC00E82FF92F06850260068705C031DE082F17
:101A0C00192F0E94301301E0899199910895F6DA0B
:101A1C0047EB5CE048DD002331F0E82FF92F068519
:101A2C0002600687F0CF1CDE082F192F0E9430139E
:101A3C00EACFE02FF12F268521FF09C0A6DEE2E4D4
:101A4C00F4E0058716872787308B01E0089500277F
:101A5C000895BFDFE2E4F4E005851685278530891B
:101A6C004185528563857485FCDB4CDE19F446E2B6
:101A7C0052E002C04FE252E0082F192F0E945C1175
:101A8C00E2E4F4E00585168527853089E82FF92FE7
:101A9C000087118722873387068502600687B3CFBC
:101AAC00ADDAB1DA01F212D041F00AD031F0E82F00
:101ABC00F92F068500680687A6CF26DEA1F7B3CFDF
:101ACC0001DE44E152E0082F192FDDCD082F192F2C
:101ADC00085F1F4F05DB012B089590DA15DE09F422
:101AEC00A2CFF4DFD9F3ECDFC9F3E82FF92F068589
:101AFC000068068788CF97CF0E94D912802FA42F19
:101B0C00B52FAEDD0A2F1B2F0E9430138823C1F096
:101B1C008830B0F400911004083091F4082F20DFC5
:101B2C0013D064F4465F5B4F0A2F1B2F11DE00238A
:101B3C0029F0EA2FFB2F06850068068701E001C01B
:101B4C000027E4E00C94EA12402F512FE05FFB4F8A
:101B5C000081003008950E94D4122F97802E442EBD
:101B6C00552E002309F476C008E0801608F072C0E8
:101B7C0000911004083009F06DC0485F5F4F0C2FC6
:101B8C001D2FE6DD002309F465C0E5E5F4E0828154
:101B9C009381A481B581CADE012B09F45BC066DB9D
:101BAC0009F458C0E42DF52D06855BDD02FF03C05A
:101BBC000385016002C003850E7F0387082F192F50
:101BCC0053D009F447C0082D4AD0202F312F065F7F
:101BDC001B4FEC2FFD2F389647E050E00E94AA12C5
:101BEC00E22FF32FE05FFB4F008100680083E42DB0
:101BFC00F52D0685205F3B4FE22FF32F02FF03C02C
:101C0C000081046002C000810B7F0083A1E0A8303A
:101C1C00F8F40A2F24D0802F912F865F9B4FE82F4A
:101C2C00F92F408051806280738099DEE65FFB4F14
:101C3C00D7D9401651066206730641F4A81531F047
:101C4C00082F192F47E050E00E94AA12A395DFCF6E
:101C5C0001E001C000272F96E9E00C94E512112752
:101C6C0047E050E00C94C4112A2F3B2FEDD90023F0
:101C7C0008959A938A93202F0023A9F0283098F482
:101C8C0000911004083079F407E01DDD5527022F70
:101C9C0047E00E94C411065F1B4F40E050E00E94D9
:101CAC00301301E001C00027899199910895002318
:101CBC0021F0083010F401E0089500270895002366
:101CCC0081F0083070F44CDEE05FFB4F0081003097
:101CDC0044F406FF03C000E011E0089500E810E0B2
:101CEC000895002711270895002379F0083068F42F
:101CFC0037DEE05FFB4F208120303CF4025F1B4F4E
:101D0C00E02FF12F008111810895002711270895EC
:101D1C000E94D5122F970FDE11274DE050E00E9444
:101D2C00C411802F912F44E152E00C2F1D2FD4DCD5
:101D3C00002309F44BC0AA2794DC848F958FA68FBF
:101D4C00A78F8EDA93DF09F441C0488459846A84E2
:101D5C007B8488279927A1E0A830B0F50A2F00DEF4
:101D6C00F3DE84F5465F5B4F0C2F1D2FF1DC002357
:101D7C0049F1042D152D262D372D7CDA39F104E48B
:101D8C002AD00A2F005D27D00DE325D0BBDC4C2FC9
:101D9C005D2F4E5F5F4F082F192F065F1D4F0E945E
:101DAC00191308960DE017D00AE015D00027E82F7C
:101DBC00F92FE65FFD4F0083042D152D262D372DB1
:101DCC0055DF21F0A395C8CF01E001C000272F9665
:101DDC00E8E00C94E612E82FF92F0196E65FFD4F30
:101DEC0000830895E6E6FF274AE050E00C94AA121F
:101DFC0005D900914204E82FF12F0083009154047F
:101E0C00018399DDE82FF92F028301E20383899185
:101E1C00999108950E94D7122F9767DA442E552E68
:101E2C0001E44ADC082F192F0E9430134A2F5B2F34
:101E3C000C2F1D2F75DC002309F459C012DC068110
:101E4C000E37D9F50E2F1F2FAA2720915F042A9544
:101E5C0020935F0491F10052104001C02EC0E02F7E
:101E6C00F12F23852F3049F5A35FA23430F5218162
:101E7C0084DC238182DC258180DC27817EDC21854A
:101E8C007CDC26857ADC208978DC228976DC248946
:101E9C0074DC268972DC208D70DC248D6EDC268D42
:101EAC00E82FF92F21938E2F9F2F22272083E02FAD
:101EBC00F12F2081203448F218C024DC08DC042DDA
:101ECC00152D0E9419130EE2E42DF52D0087D3DB9E
:101EDC00FEDB485F5F4F042D152D075F1F4F0E94DF
:101EEC0019130027E42DF52D048701E001C000270C
:101EFC002F96E6E00C94E8120E94CF12802EA42EAE
:101F0C00B52ECE84DF84002309F463C008E080166C
:101F1C0008F05FC024DDE05FFB4F808180300CF067
:101F2C0058C01DDDE25FFB4F008111810A151B05B6
:101F3C0008F44FC00A2D0B2909F44BC086FF04C0CE
:101F4C00662401E0702E03C000E8602E772445D093
:101F5C000A2D1B2D0FD80A2D1B2D1FDA71F08AD9D3
:101F6C00C1F10A2D1B2D0DDA005F1F4F7A926A9278
:101F7C00065F1D4F402F512F26C07CD951F100E137
:101F8C0012E006191709262D372D205130403A93AF
:101F9C002A93065F1D4F402F512F0C2D1D2D0E9493
:101FAC0019138F5F9F4FAF4FBF4F60D991F0062D24
:101FBC00172D0051104020E130E03A932A934AE06B
:101FCC0052E0C00ED11E0C2D1D2D0E94191301E0E4
:101FDC0001C00027E0E10C94E01200E012E0462D75
:101FEC00572D0E94E211402E512E08950E94CD12C1
:101FFC00802EC42ED52EE888F988002309F46BC0F6
:10200C0008E0801608F067C0AADCE05FFB4F808117
:10201C0080300CF060C082FD5EC0A1DCE25FFB4F43
:10202C00008111810C151D0508F455C00C2D0D29CE
:10203C0009F451C086FF04C0662401E0702E03C071
:10204C0000E8602E7724C9DF0C2D1D2D0E94C007DF
:10205C00882E992EAA2EBB2E0C2D1D2D9ED991F0BB
:10206C0009D9C9F10C2D1D2D8CD9802F912F40969B
:10207C007A926A9234D00E941913082D192DF4DD2E
:10208C0051F127C0F7D839F180E192E08619970910
:10209C00062D172D005110401A930A9320D0FEDA0A
:1020AC00E5DDC9F00FEF801A900AA00AB00A862D60
:1020BC00972D80519040F4DADDD869F000E103DB14
:1020CC00E80EF91E4E2D5F2D0AE012E0E7DACEDDA8
:1020DC0011F001E001C00027E2E10C94DE124E2D5C
:1020EC005F2D865F9D4F082F192F08950E94D812DF
:1020FC002A97A02FB12F44E152E0EEDA002309F425
:10210C0074C0EA2FFB2F04851585012B09F06DC0D7
:10211C0078D00AE014E06ED00E94F407ABD809F432
:10212C0064C0FBDB0AE012E00E948211802F912F29
:10213C00012B09F45AC0E82FF92F0081043409F05F
:10214C0044C002810D3309F040C0418000ED400EC7
:10215C00E1F108E04016C8F5082F192F0D5F1F4F4D
:10216C000E9441130930104080F5CCDA40E250E077
:10217C000C2F1D2F0E5F1F4F0E943013082F192F8D
:10218C000D5F1F4F0E9441131A930A930396482F19
:10219C00592F0C2F1D2F0E5F1F4F0E9419134C2F00
:1021AC005D2F0A2F1B2FC8DA002379F00A2F1B2F63
:1021BC00BFDB012B29F0EA2FFB2F06850068068771
:1021CC00042D4DDD065F1B4F15D00E94F40752D82D
:1021DC0061F0A3DB002711270E948211802F912F21
:1021EC00012B09F0A8CF01E001C000272A96E5E0F9
:1021FC000C94E912EA2FFB2F389647E050E00C9430
:10220C00AA1208E359DA0AE014E00C943013609730
:10221C0003E152DA02E414E00E943013F2DF06E626
:10222C0011270E944105002361F0B4DA002349F024
:10223C000C2F1D2F0F5F1F4F59DF002311F001E0F2
:08224C0001C00027609608950F
:04023800FFFFFFFFC6
:100210004154520053494F32494445200043464718
:100220000020090D0A00433A28524F4F5429002854
:080230005355424449522900D4
:1022540028813981622F732F21503040672BD9F0A8
:10226400E02FF12F6081E42FF52FC895601571F0F0
:10227400E02FF12F0081E42FF52FC895001618F4F4
:1022840001E010E00AC00FEF1FEF07C00F5F1F4F00
:102294004F5F5F4FDFCF002711272296089505D0A7
:1022A4000F5F1F4F008311830895E82FF92F0081DA
:1022B400118108959A938A938A819B81282F392FBB
:1022C4000197232B59F0E42FF52F4F5F5F4FC895EB
:1022D400E02FF12F01920E2F1F2FF0CF89919991AA
:1022E40022960895E02FF12FC895002031F0C8956B
:1022F400041629F00F5F1F4FF5CF0027112708950B
:102304000E94D712442E552E8E819F81202F212B7F
:1023140021F0E82FF92F00831183C7DF012B41F04F
:102324002BD021F020D011F0BADFFACF25D019F448
:102334000027112715C0E82FF92FA081B1811CD0E7
:1023440069F011D011F4ABDFFACF0027E82FF92F91
:1023540020813181E22FF32F0083A1DF0A2F1B2F6D
:10236400E8E00C94E812A1DFE02FF12F4081042D66
:10237400152DB8DF012B089598DFE02FF12F008190
:042384000023089595
:10238800002411240030010741F01695079510F438
:10239800040E151E440F551FF5CF002D112D08955D
:0E23A8004A9522F0000F111F0C94D4110895D5
:0E23B6004A9522F0169507950C94DB110895B8
:1023C40000241124E0E1EA9552F0001F111F001CC3
:1023D400111C04161506B8F3041A150AF4CF001FCD
:0C23E400111F402D512D009510950895FB
:1023F0000024112422243324E02FE12BE22BE32BB1
:1024000071F0369527951795079520F4040E151E43
:10241000261E371E440F551F661F771FEDCF002D58
:08242000112D222D332D08952A
:102428004A9532F036952795179507950C9414120E
:02243800089505
:10243A000024112422243324E0E2EA9592F0001FBA
:10244A00111F221F331F001C111C221C331C0416CF
:10245A0015062606370688F3041A150A260A370AC5
:10246A00ECCF001F111F221F331F402D512D622D4B
:0C247A00732D0095109520953095089565
:10248600C895702D3196C895602D3196C895502DFA
:102496003196C895402D3196C8953196102C01FA83
:1024A600C8953196202CC8953196302C0895F1DFC9
:1024B600041B10E003C0EADF041B150B20E030E02C
:1024C60005C0DEDF041B150B260B370BC8F010FC0E
:1024D6001AC03AD0402D38D00417100588F446F4B7
:1024E600E00FF11FC895E22DF32DE019F040099495
:1024F600000F111FE00FF11F27D0202C25D0302C04
:10250600E22DF32D099411F4BEF7ECCF31960EF0BF
:10251600319650E060E070E017D0402D4B3F68F0F8
:1025260079F34F3F41F04E3F21F00ED0702D0CD085
:10253600602D0AD0502D08D0402D041B150B260BFC
:0E254600370B11F3E8F2E2CFC89531960895F5
:10255400BF93AF93A02FB12F02C001900D924150B1
:0A2564005040D8F7AF91BF910895E1
:10256E00BF93AF93A02FB12F03C0C89531960D9294
:0C257E0041505040D0F7AF91BF9108953C
:0E258A00002401C0019201501040E0F70895B6
:02259800000041
:10259A00FA92EA92DA92CA92BA92AA929A928A9291
:1025AA007A926A925A924A92BA93AA939A938A937D
:0225BA00089582
:1025BC00FF84EE84DD84CC84BB84AA8499848884D3
:1025CC007F806E805D804C80BB81AA8199818881DF
:0E25DC00F0E00FB6F894CE0FDF1F0FBE08958B
:1025EA0028813981622F632B79F0E02FF12F6081E6
:1025FA00E42FF52F7081671739F40F5F1F4F4F5F74
:10260A005F4F21503040EECF232B51F0E02FF12FB6
:10261A0000811127E42FF52F2081021B104002C0F0
:08262A000027112722960895F4
:1026320068817981202F312F062E172E615070402C
:10264200012859F0E42FF52F0080E22FF32F019299
:0E2652002E2F3F2F4F5F5F4FEFCF2296089540
:102660009A938A938A819B81E02FF12F282F392F0B
:102670000197232B11F04193F9CF899199912296DB
:022680000895BB
:10268200E02FF12F2081222311F03196FBCFE01BA6
:08269200F10B0E2F1F2F08951C
:00000001FF
